:1000000047C15FC15EC15DC1EEC15BC15AC140C2A3
:1000100058C157C156C155C10AC2BCC152C151C114
:1000200050C14FC14EC14DC14CC114641E006E146D
:10003000001E503C057F0500147812036455041E11
:100040007F000078050000000000000000040F7D24
:100050000A326400043264001E780A04235A05142C
:100060006400000000000000000F000A7F0014641C
:100070000A052846000A3C0A00087805785A0C0050
:100080005F19000064000000000000000A505005E5
:10009000465A050A5A3C0041500A0A64640A50460E
:1000A000050000000000000004007F00007F001435
:1000B0001E5A000064140464320064320000000020
:1000C000000000000864640F64640F08503C055091
:1000D0003C0504321403321403040A0A0F0A0A0FFF
:1000E0000802052802052808060A1E060A1E020A3A
:1000F0000A0F0A0A0F0632140332140304503C0597
:10010000503C05000000000000000A3250643C50E2
:100110005A0A283C503250640A1E3C5A283C500A65
:100120000A28461E3C5A0A3C505A0A28460000003B
:10013000000000000A78285A78285A056E1E0A64C2
:1001400028050A32147F32147F00000000000000EE
:100150000A190008170005375A00005A0000081E47
:1001600000001E0000077878007878000A1E000062
:100170001E00000A7F14007F140000000000000031
:1001800000047F0000007F0004007F007F0000006B
:10019000000000000000041E280000007F045A78C0
:1001A0000000003200000000000000083C00003C9D
:1001B00000000823370023370008005A00005A00C7
:1001C000080041550041550800007F00007F0823CA
:1001D000003723003700000000000000046E7F009D
:1001E000000000040000006E7F000000000000001E
:1001F00000040006080006080250785A50785A0297
:1002000000060800060800000000000000C8000A00
:1002100028000A285000143C00194178000F2C00D7
:100220000A28280014500014500A00051400021770
:10023000017F7F7F7F7F7F01000514000217280068
:10024000143C000A3278000F32000822000000003F
:100250000000002A00610F4D00C21E6900610F8C72
:10026000001303A800C21EC40010F60A01270634BA
:1002700001C21E500113038101CA999601CA99ABAC
:1002800001CA99DC01C21EF101C21E0D0213030056
:1002900011241FBECFEDCDBF10E0A0E6B0E0EAED27
:1002A000F7E002C005900D92A638B107D9F710E02B
:1002B000A6E8B0E001C01D92A13BB107E1F780D1F3
:1002C0008AC29ECE0F931F93CF93DF93282F392F8F
:1002D00006E810E0ACE8B0E0E2E9F0E0862F972F06
:1002E00071E061ECE90159919E0157FD5FE7EC0176
:1002F0004991CE0147FD4FE7541724F4451B4C9319
:10030000708303C0541B5C931082E80169938E01D3
:100310001196319640E0CC38D40721F78FE78093CF
:100320009800DF91CF911F910F910895EF92FF9266
:10033000CF93DF93E6E8F0E04CE850E0E82EE701E9
:100340007E01F92EE70182E990E0DA012D91AD01FD
:100350003081230F2083121664F4DC013C91288144
:10036000332311F02F5F01C02150288320812F57A4
:100370002083319621960196B0E0EC38FB0729F7EF
:1003800080919800815080939800DF91CF91FF90E9
:10039000EF9008951F920F920FB60F9211242F9392
:1003A0003F934F935F936F937F938F939F93AF93FD
:1003B000BF93EF93FF9382EA90E0A5D198B3907C2E
:1003C000982B98BBFF91EF91BF91AF919F918F9127
:1003D0007F916F915F914F913F912F910F900FBE41
:1003E0000F901F9018951F920F920FB60F92112425
:1003F0002F933F938F939F938AB59BB520919E0037
:1004000030919F00820F931F9BBD8ABD8091AE00EB
:1004100090E0009719F001978093AE009F918F9123
:100420003F912F910F900FBE0F901F9018951F9224
:100430000F920FB60F9211242F938F939F9388B52D
:1004400099B5805E914B99BD88BD20B320952077EA
:1004500041F48091A0009091A1008230910520F09C
:1004600002C08CED95E001979093A1008093A000CD
:1004700080919A00882311F42093990020939A0088
:100480009F918F912F910F900FBE0F901F901895F5
:100490001F920F920FB60F9211242F933F934F93F9
:1004A0005F936F937F938F939F93AF93BF93EF93DC
:1004B000FF934CD1FF91EF91BF91AF919F918F919D
:1004C0007F916F915F914F913F912F910F900FBE50
:1004D0000F901F90189581B38F7881BB82B380678E
:1004E00082BB87B38F6387BB88B3807C88BB82E085
:1004F00080BF83BF93E396BF1FBC8EBD82EC9EE19D
:100500009BBD8ABD80E29EE499BD88BD81E689BF1E
:100510000895A82FB92F80E090E00196FB01E80F25
:10052000F91FE491ED9386309105B9F70895EF92A4
:10053000FF920F931F93CF93DF938C01EB012097D2
:1005400051F482EA90E0B801E4DFE02EE7017E0199
:10055000F12EE7010EC088EA90E0DBDF82EA90E04E
:1005600068EA70E0AFDEFE01849180939D00809385
:10057000AE002796FE018491882329F4E02EE7013E
:100580007E01F12EE701CE01DF91CF911F910F91F6
:10059000FF90EF90089590E0880F991F880F991FA2
:1005A000FC01EB5AFD4F2591349120939E0030932E
:1005B0009F008D5A9D4FFC0125913491C9010895EA
:1005C000DF92EF92FF920F931F93CF93DF9383DF1E
:1005D000B4D080E090E0DCD0F82E8F3028F080E0BE
:1005E000DADFEC01FF2409C0D6DFEC0182E090E005
:1005F000CFD090939F0080939E00CE0160E070E08A
:1006000096DFBC01CE0193DF8C017894EE24EA944E
:1006100052E0D52E809199008032F1F0803419F0AB
:10062000803161F510C0E092990080919E00909118
:100630009F008E399105C0F09695879590939F0005
:1006400080939E001BC0E0929900FF2011F0FA9465
:100650000BC03EE0F32E08C0E09299008F2D8E3043
:1006600011F0F39401C0FF248F2D95DFEC0160E0C1
:1006700070E05DDFBC01CE015ADF8C0180919C00EF
:10068000882389F48091AE00882369F480919D00CD
:100690008093AE0082EA90E049DE882321F4CE0107
:1006A000B80145DF8C0180919C00813099F4E09184
:1006B000AF00E254E63228F4F0E0E05AFF4FE08168
:1006C00001C0E0E0F0E0EE55FF4F8091B000808384
:1006D000D0929C008091A0009091A1008130910562
:1006E00009F098CF80E090E06F2D70E054D06091D9
:1006F0009E0070919F0082E090E04DD01092A1008A
:100700001092A00087CF9C0180919B00882311F05C
:10071000815001C08EE780939B0040919B0080E058
:1007200096E09150880FF901E90FF11D50814517AE
:1007300008F481609923A9F708951BB880E98AB964
:1007400086E083B912B88FEC89B908958CB18134F1
:1007500028F08093AF001092B0000CC08D3051F49F
:100760009091AF00983719F410929C0003C091E06B
:1007700090939C00982F90539A3048F48091B00049
:10078000880F980F880F880F980F9093B0000895E6
:10079000A8E142E005C011D0272F10C0A82F862F56
:1007A000E82FE199FECF1FBA05C0EEBBE09AE395B2
:1007B0000DB20D924150C8F70895262FE199FECF52
:1007C0001CBA1FBA8EBB2DBB0FB6F894E29AE19A01
:0A07D0000FBE01960895F894FFCFC4
:1007DA000500000000040000000000000000000006
:1007EA0003000000000000000000000000000000FC
:0607FA00020000000001F6
:00000001FF
